:020000040800F2
:10000000C825002025020008F9020008F1020008B6
:10001000F5020008E1020008950300080000000056
:100020000000000000000000000000002D03000898
:10003000E502000800000000290300083103000861
:100040003F0200083F0200083F0200083F0200088C
:100050003F0200083F020008E90200083F020008D2
:100060003F0200083F0200083F0200083F0200086C
:100070003F0200083F0200083F0200083F0200085C
:100080003F0200083F0200083F0200083F0200084C
:100090003F0200083F0200083F0200083F0200083C
:1000A0003F0200083F0200083F0200083F0200082C
:1000B0003F0200083F0200083F0200083F0200081C
:1000C0003F0200083F0200083F0200083F0200080C
:1000D0003F0200083F0200083F0200083F020008FC
:1000E0003F0200083F0200083F0200083F020008EC
:1000F0003F0200083F0200083F0200083F020008DC
:100100003F0200083F0200083F0200083F020008CB
:100110003F0200083F0200083F0200083F020008BB
:100120003F0200083F0200083F0200083F020008AB
:100130003F0200083F0200083F0200083F0200089B
:1001400000000000000000000000000000000000AF
:100150003F0200083F0200083F0200083F0200087B
:100160003F0200083F0200083F0200083F0200086B
:100170003F0200083F0200083F0200083F0200085B
:100180003F02000800F002F800F03CF80AA090E8F6
:10019000000C82448344AAF10107DA4501D100F042
:1001A00031F8AFF2090EBAE80F0013F0010F18BFD3
:1001B000FB1A43F001031847884E0000A84E0000C8
:1001C000103A24BF78C878C1FAD8520724BF30C883
:1001D00030C144BF04680C60704700000023002455
:1001E00000250026103A28BF78C1FBD8520728BF47
:1001F00030C148BF0B6070471FB501F07FFA1FBDCB
:1002000010B510BD00F031F81146FFF7F5FF01F011
:1002100063F800F04FF803B4FFF7F2FF03BC00F0FF
:1002200057F800000948804709480047FEE7FEE705
:10023000FEE7FEE7FEE7FEE7FEE7FEE7FEE7FEE796
:1002400004480549054A064B70470000350300087D
:1002500085010008C81F0020C8250020C8210020F3
:10026000C8210020704770477047754600F02CF891
:10027000AE4605006946534620F00700854618B093
:1002800020B5FFF7DDFFBDE820404FF000064FF03E
:1002900000074FF000084FF0000BAC46ACE8C00977
:1002A000ACE8C009ACE8C009ACE8C00921F007011E
:1002B0008D46704710B50446AFF300802046BDE878
:1002C0001040FFF7A8BF000000487047080000205A
:1002D00001491820ABBEFEE726000200704700006F
:1002E000FEE700007047000080B500F0F1F880BD27
:1002F000FEE70000FEE700007047000000F0070086
:1003000080F00703042B28BF04234FF0FF3C033881
:100310000CFA03F338BF0020994381400CFA00F037
:1003200022EA000008437047704700007047000051
:10033000704700004EF6885CCEF2000CDCF800201E
:1003400041F2000142F47002C4F20201CCF8002034
:100350000A6842F001020A600A689207FCD54A68FE
:1003600022F003024A6000BF4A6812F00C0FFBD172
:1003700000224A600B684FF6FF70CFF6F26018401B
:1003800008604FF41F000A6388604FF000604CF86B
:10039000800C7047FEE70000002848BF704700F05F
:1003A0001F01012202FA01F14EF200124009CEF2C1
:1003B000000242F8201070474EF60C50CEF20000BA
:1003C0000068C0F3022070474EF6145300F00F028D
:1003D000CEF2000309011A4400F16043B0F1FF3F7F
:1003E000C8BF03F564421170704700004EF60C510F
:1003F000CEF200010A684FF6FF031A4060F30A22AA
:1004000042F0806040F0FD7008607047B0B543F680
:1004100000050446C4F200052846022101F058F800
:100420000028F9D02846214601F050F8B0BD000060
:1004300010B543F60004C4F2000400BF204680213A
:1004400001F046F80028F9D110BD000070B584B065
:100450004FF4C0100121012500F0FAF8002000211E
:10046000002600F063FE01AC204600F00BFE40F2D7
:100470000110ADF80C0020468DF80460029500F0E4
:100480000DFE032001F00CF806200021002200F0F0
:10049000F5FF04B070BD0000B0B582B00220C0F21C
:1004A00018000121012500F0D3F86C46204600F029
:1004B00033FE41F60000C0F20010CDE9005040F6D6
:1004C0000000C4F20100214600F076FE02B0B0BD8B
:1004D00080B5052000F054F9012000F0D9FD40F668
:1004E0000000C4F20100012100F0C6FE002818BF80
:1004F00080BD40F20000C2F200000178042204290D
:1005000008BF0122027080BD41F20401C4F2020161
:100510000A6800F00F0022F0F00242EA00100860C2
:100520007047000041F20401C4F202010A6800F0C1
:10053000070022F4E06242EA0020086070470000F1
:1005400041F20401C4F202010A6800F0070022F43B
:10055000605242EAC02008607047000041F2540136
:10056000C4F202010A68012822F0300208BF3032CA
:100570000A607047042888BF7047DFE800F0030C6A
:1005800019262F0041F20000C4F20200026861F354
:1005900000020260704741F20000C4F202000268EB
:1005A00001F0010122F4803242EA0141016070470A
:1005B00041F20000C4F20200026801F0010122F0E1
:1005C000807242EA01610160704741F20000C4F2AA
:1005D0000200026A61F300020262704741F2000009
:1005E000C4F20200426A61F30002426270470000F6
:1005F00041F20002010CC4F20202895800F01F000F
:1006000021FA00F000F001007047000041F25401AF
:10061000C4F202010A6800F0030022F4405242EAE8
:10062000003008607047000010B500241120FFF76B
:10063000DFFF210B022903D8012804F10104F5D1C1
:100640001120FFF7D5FF0138B0FA80F0400910BD46
:1006500041F2000200F01F034FF0010CC4F202024D
:1006600001290CFA03F14FEA1040835814BF23EA22
:10067000010119438150704780B541F2040EC4F264
:10068000020EDEF800C060B14CF48033CEF80030CA
:10069000DEF800C0012814BF4CF400302CF4003008
:1006A00001E02CF48030CEF80000DEF8000061F3A9
:1006B0009540CEF80000DEF80000C1F3021161F3AE
:1006C0005E70CEF80000DEF8000020F0004040EA46
:1006D000C270CEF8000080BD41F20000C4F20200FA
:1006E000016841F00101016001688907FCD541689A
:1006F00021F00301416000BF416811F00C0FFBD1F4
:100700000021416002684FF6FF73CFF6F2631A4092
:10071000026001634FF41F018160704741F20401E0
:10072000C4F202010A6860F301020A607047000027
:1007300041F20400C4F202000068C0F38100704777
:1007400080B5042000F0CEFF40F20400C2F20000A9
:1007500000684DF68361C4F21B31A0FB0101880CD7
:1007600040F28001C2F20001086008684FF47A711B
:10077000484340F27C01C2F20001086080BD0000E5
:1007800080B5002808BF80BD4EF2100140F27C0EFB
:10079000CEF20001C2F2000E4FF0320C002300BF77
:1007A00082B2332A06D3DEF80020323802FB0CF284
:1007B0004A6004E0DEF800005043486000208B608F
:1007C0000A6842F001020A600A6802F00112012A76
:1007D000FAD00A6822F001020A6002048B60DFD1BD
:1007E00080BD000080B540F60040C4F201004FF427
:1007F000805100F08DFC80BD80B540F60040C4F211
:1008000001004FF4805100F085FC80BD80B540F6BA
:100810000040C4F201004FF4804100F079FC80BD3B
:1008200080B540F60040C4F201004FF4804100F072
:1008300071FC80BD80B5FFF7A3FF80BD2DE9F043BB
:1008400081B08846054600200021002600F0B0FB5C
:10085000242000F0FDFBFFF7C5FFA5F101090027EB
:1008600009EB0605002400BF15F8010FFFF7CEFDC8
:10087000013C14F1FA00F7D10137102FA6EB040662
:10088000EED1FFF7D5FDFFF7B7FF002000210025CF
:1008900000F08EFB262000F0DBFBFFF7A3FFA8F1A2
:1008A0000108002608EB0504002700BF14F8010F1B
:1008B00080F0FF00FFF7AAFD013F17F1FA00F5D124
:1008C0000136102EA5EB0705ECD1FFF7B1FDFFF7C0
:1008D00093FF00F087FB01B0BDE8F08310B504463C
:1008E000102000F0B5FB204600F09CFB10BD00007E
:1008F00080B500F049FB3220FFF79CFF00F04EFB73
:100900003220FFF797FF00F07BFB28B9122000F0A0
:100910009FFB00F075FB08B1012080BD012000F0B5
:1009200097FB272000F07EFB012000F07BFB0120DD
:1009300000F078FB112000F08BFB012000F072FB2F
:10094000442000F085FB002000F06CFB0F2000F03D
:1009500069FB452000F07CFB272000F063FB0120B1
:1009600000F060FB002000F05DFB002000F05AFB6F
:100970003C2000F06DFB052000F054FB212000F02E
:1009800067FB002000F04EFB802000F04BFB18209E
:1009900000F05EFB802000F045FB4E2000F058FB8D
:1009A000002000F03FFB4F2000F052FB272000F01A
:1009B00039FB012000F036FB00F022FB002818BFB5
:1009C000012080BD2DE9F04184B00224C0F218045A
:1009D00020460121FFF73CFE601C0121FFF738FE95
:1009E00002AD284600F098FB40F60044C4F2010432
:1009F000A4F5806630464FF480714FF4807700F0A4
:100A000087FB40F20040C0F21010CDE90270304682
:100A1000294600F0D1FB1820ADF80D004FF400700E
:100A200002903046294600F0C7FB20464FF4804133
:100A30004FF4804600F06EFB4FF010084FF48067D3
:100A4000204629468DF80E80ADF80C70029600F015
:100A5000B3FB4FF400500826029020462946ADF81B
:100A60000C708DF80E6000F0A7FB4FF40040029070
:100A7000204629468DF80E6000F09EFB20464FF47C
:100A800080514FF4805600F045FB204629468DF8F2
:100A90000E80ADF80C70029600F08EFB0E20C0F2B6
:100AA0001C000121FFF7D4FD6D46284600F0FCFC38
:100AB00040F20310C0F20500009040F20010C0F2B6
:100AC0000110A4F5544401902046294600F006FD8B
:100AD0002046012100F0F0FC04B0BDE8F0810000E8
:100AE00080B540F60000C4F201004FF4007100F040
:100AF000C3FB002818BF012080BD000080B540F274
:100B0000680CC2F2000CBCF81210002908BF80BDAE
:100B10004FF0000E06E000BFBCF812100EF1010EFF
:100B20008E4512D2BCF81030002BF5D04FF0FF31BB
:100B3000DCF800200EFB03220A445070BCF8103091
:100B40008A1C01319A42F3D3E6E780BD2DE9F04FCC
:100B500085B006461046B2EB060B0F46049248BF1E
:100B6000CBF1000BD81B80EAE071024648BF42423D
:100B7000C1EBE07904984FF0FF31B0424FF0FF38FD
:100B8000ABEB020A88BF4FF0010818460293BB4244
:100B900088BF01210191039203E000BFBBEB4A0F24
:100BA00011DAB4B2BDB20E9A2046294600F016F80A
:100BB000B9EB4A0FF2DC049884420BD00398464408
:100BC000AAEB000AEAE70298854203D00198DA44CA
:100BD0000744E6E705B0BDE8F08F000080B50138B6
:100BE000013980B289B200F06FF880BD2DE9F04183
:100BF00082B00F46DDE908811C461546064681B1E4
:100C0000A7420BD2B9B230462A460B46CDF8008037
:100C1000FFF79CFF0137B8B2A042F3D302B0BDE8A2
:100C2000F081304639462A463B46CDF80080FFF732
:100C30008DFF3046394632462346CDF80080FFF717
:100C400085FF284621462A463B46CDF80080FFF71F
:100C50007DFF2846214632462346CDF80080FFF727
:100C600075FF02B0BDE8F08110B540F2680CDDF808
:100C700008E0C2F2000CCCF80000C8084C07ACF841
:100C80000810ACF80A20ACF80CE04FF0010E18BFC9
:100C90000EEBD100ACF81000ACF81220ACF80E301E
:100CA0002BB1B42B12BF084610460A4601E010468D
:100CB0000A46ACF80400ACF8062010BD40F268010A
:100CC000C2F200010860704710B540F2680CC2F231
:100CD000000CBCF80E30B32B0BDC93B15A2B36D181
:100CE000BCF80830C0431844BCF80A30C9435C184B
:100CF00013E0B42B0CD0B3F5877F0C4618BF10BDA2
:100D00000BE0BCF808E0C94304460EEB010004E028
:100D1000BCF80A30C0431C180846BCF81030A4B216
:100D200081B26343DCF800C003EBD10E1CF80E3037
:100D300000F007008024C4401C436FF0800141FA9A
:100D400000F0002A08BF03EA00040CF80E4010BDB2
:100D50002DE9F04F87B00130039080B20290C01AA5
:100D6000FA2800F38380082B02D1062464B97DE0C1
:100D7000D8085F074FF0010618BF06EBD3005F08E5
:100D8000784384B2002C71D04E1C109DA2F120003B
:100D900041F6B25182B25808C0F60001DDF80C905D
:100DA000B5FA85F70190002001EB02114FF0000821
:100DB00004920091CDE9054312E000BF02991FFAA9
:100DC00089F0401A019926468842039804BF81465B
:100DD0000836059908F101081FFA88F0814245D9C3
:100DE000082B09D1049941F2167201EB4101C0F6BA
:100DF000000202EB410119E0182B0BD0102B13D08D
:100E00000C2B33D1049941F63E1201EB4101C0F69F
:100E1000000206E0049942F2A23201EBC101C0F6E1
:100E2000000202EB810101E0009900BF084490F844
:100E300000A04FF0000B34465FEACA702A461FFA42
:100E400089F0B1B208BF7A09FFF7C8FE4FEA5A0A23
:100E50000136BBF1070F0BF1010BEDD3069B09F136
:100E60000109082BAAD105992646B3E707B0BDE8CA
:100E7000F08F00002DE9F04F87B0DE085F07059284
:100E80004FF0010218BF02EBD306002E009653D09C
:100E9000119E00F1010A4A1CB6FA86F51FFA8AF083
:100EA00000234FF0000B17460390CDF810A004E08C
:100EB0000133009998B288423ED205980028F7D0B5
:100EC0004FF000080293CDF804B000BF10991FFA4C
:100ED0008BF00C5C4FF00009069200BFE007324631
:100EE0001FFA8AF0B9B218BF6A09FFF777FE6408E3
:100EF0000137B9F1070F09F10109EFD30AF1010A2E
:100F000003991FFA8AF0401A059908F101088842EE
:100F1000049808BF8246069A1FFA88F00BF1010B6D
:100F200008BF083288421746D0D30598DDF804B0D0
:100F3000029B83441746BBE707B0BDE8F08F000073
:100F40002DE9F04381B099461378CBB1DDF82080CC
:100F50000D4606464FEA5907541EB9F1080F08BF5F
:100F6000062700BFB0B2DAB229464B46CDF8008062
:100F7000FFF7EEFEA3783E44002B04F10104F1D10B
:100F800001B0BDE8F083000080B540F60000C4F277
:100F900001004FF4807100F0BBF880BD80B540F6D1
:100FA0000000C4F201004FF4807100F0B3F880BD7E
:100FB000B0B5044640F22710451A4E20F92988BFE3
:100FC0002E2500F045F8C4F3C70000F02BF84F20A1
:100FD00000F03EF8E8B200F025F8C5F3002000F07C
:100FE00021F8B0BD80B5222000F032F8F72000F0E3
:100FF00019F8202000F02CF800F002F880BD000065
:1010000010B5FFF76DFD58B144F621640120013C95
:1010100008BF10BDFFF70EFCFFF762FD0028F5D1F9
:10102000002010BDB0B543F600040546C4F200042C
:10103000FFF7D8FB2046294600F048FA20468021D9
:1010400000F046FA0028F9D1FFF7D6FBB0BD00004A
:10105000B0B543F600040546C4F20004FFF7D6FB22
:10106000FFF7C0FB2046294600F030FA20468021D9
:1010700000F02EFA0028F9D1FFF7BEFBFFF7D0FBF6
:10108000B0BD000000214160012101810170704765
:1010900040F21441C4F201010860704740F2084177
:1010A000C4F20101426851F8083C934341F8083CFE
:1010B00051F8043C934341F8043C437A002B08BFA9
:1010C000704703786FEA020C2BB151F8043C1343CC
:1010D00041F8043C04E051F8083C134341F8083C53
:1010E0000B6803EA0C030B604B6803EA0C034B60CC
:1010F000007A012807D018B90868104308607047C3
:101100000868104308604868104348607047000052
:10111000416170470161704740F200424FF6FF7134
:10112000C0F20012C0E900127047000080B58B08C1
:10113000032B88BF80BD0C2202EA810E4FF00F0CFA
:1011400002EB83010CFA0EF2DFE803F002290F1C18
:101150000821C4F201010B6800FA0EF023EA020232
:101160000A600A681043086080BD0821C4F20101CA
:101170008B6800FA0EF023EA02028A608A68104344
:10118000886080BD0821C4F20101CB6800FA0EF02E
:1011900023EA0202CA60CA681043C86080BD082101
:1011A000C4F201014B6800FA0EF023EA02024A6021
:1011B0004A681043486080BDB0B58B790A88032B1C
:1011C0000BD07BB94979282901F00F0E18D01829C6
:1011D00008BF0261110616D12EE04FF0000E110675
:1011E00011D129E003F0080C0B79C97903F004034D
:1011F000634401F0030103EB010E110603D11BE070
:101200004261110618D000234FF00F0C002104E0BA
:101210000131082903F104030ED022FA01F4E40796
:10122000F6D004680CFA03F5AC43046004680EFAC7
:1012300003F52C430460EBE7B2F5807F38BFB0BD07
:10124000120A00234FF00F0C002104E0013108299D
:1012500003F104030ED022FA01F4E407F6D0446847
:101260000CFA03F5AC43446044680EFA03F52C43D2
:101270004460EBE7B0BD000080680840401AB0FA57
:1012800080F040097047000010B582B00420C0F221
:1012900018000121FFF7DCF96C462046FFF73CFF00
:1012A00040F20040C0F2101001904FF40050009046
:1012B00041F20000C4F201002146FFF77DFF02B0B9
:1012C00010BD000041F20C00C4F20100016881F47D
:1012D000005101607047000088B000F075F9FFF719
:1012E0002FFAFFF7D9F8FFF7B1F8FFF7CDFFFFF7B7
:1012F00069FBFFF7FDFA40F28404C2F20004FF2705
:1013000020467A21FA22B4230097FFF7ADFC41F280
:101310002405C2F2000528467A21FA22B423009758
:10132000FFF7A2FC2046FFF7C9FCFF20FFF7E6FB12
:1013300043F2FE00C0F600000026009000200021CD
:10134000FA227A230196FFF795FD2846FFF7B6FCAF
:10135000FF20FFF7D3FB44F29E00C0F60000009090
:1013600000200021FA227A230197FFF783FD20460F
:101370002946FFF763FA4FF4FA50FFF701FA2046C7
:10138000FFF79CFCFF20FFF7B9FB29A20A200021F0
:1013900018230096FFF7D4FD2AA20A201D2110234E
:1013A0000096FFF7CDFD2EA20A20322110230096D1
:1013B000FFF7C6FD2846FFF781FCFF20FFF79EFBE5
:1013C00046F26C40C0F22E00069045F22070C7F243
:1013D0006F20059046F66540C6F66C70049043F6A3
:1013E0003E60C4F62000039003AA0A204721182378
:1013F0000096FFF7A5FD01270A206721F02274233C
:1014000000960197FFF7F2FB20462946FFF716FAF0
:101410000120FFF763FA40F20004C2F200046425E1
:10142000FFF750FF20786843FFF7AAF9F8E700BFFD
:10143000322E313320457061706572204D6F6475B6
:101440006C65000044657369676E656420427920AD
:1014500057654163742053747564696F0000000020
:10146000776974682032353020782031323220722A
:1014700065736F6C7574696F6E00000070B514460B
:101480000D460646FEF798FF29462246FEF736FF30
:1014900001463046FEF798FF3046FEF77DFF70BDEF
:1014A00080B5FEF7A3FF80BD0021C0F803100160E6
:1014B0000121C17170470000026801F0010122F0B2
:1014C000400242EA8111016070470000C16070472C
:1014D0008068084018BF012070470000C26922F4EC
:1014E0000062C2610A78032A27D8DFE802F0020608
:1014F000121A026822F400420EE0026822F400424E
:101500000260026822F480420260026842F4806253
:1015100012E0026842F400420260026822F4804253
:1015200006E0026842F400420260026842F480422F
:101530000260026822F480620260CA79036802F0E5
:10154000010223F4007343EA422202604A78012A2E
:1015500006D1CA79012A03D1026842F4807202E0FE
:10156000026822F4807202604A78036862F38203A0
:1015700003608A784368072A23F4807388BF03F5E1
:10158000807343608A78036862F3C5030360CA7896
:10159000036802F0010223F0800343EAC2120260F2
:1015A0000A79036802F0010223F4006343EAC222CD
:1015B00002604A79036862F3410303608979026833
:1015C00061F300020260704780B5FFF785F80120E3
:1015D0000121FEF7CFFF00BFFFF726F80028FBD060
:1015E00002203B210122FFF747F80020FFF70EF809
:1015F00002200121FEF7BEFF1920FEF7F9FF0128A6
:10160000FAD10020FEF780FF0420FEF799FF0420A6
:10161000FEF788FF0120FEF7A1FF0220FFF77EF80A
:10162000FFF786F80228FBD10020FEF797FF00F0B5
:1016300001F880BDB0B541F2040441F20025C4F2C6
:101640000204C0F27A05FFF773F802280BD090BBB2
:10165000206D80052FD5E06A800144BF46F6004525
:10166000C0F2DC2527E0206821682268C1F38341AD
:10167000C2F3417213010133002A1A4608BF022245
:101680000F2908BF1A46C00302EB010006D440F63A
:101690000011C0F23D0100FB01F50CE02168890357
:1016A00001D4454307E0216DC1F301310231B5FB9F
:1016B000F1F101FB00F540F20400C2F20000056008
:1016C000216804A2C1F30311515C026822FA01F1FE
:1016D0000160B0BD00000000000000000102030432
:1016E000060708094EF21001CEF200010A6804282C
:1016F00022F0040208BF04320A607047F1EE100ABB
:101700004FF6FF71C0F2C03120EA010040F0407096
:10171000E1EE100A70470000000000000000002FFA
:10172000000000000700070000147F147F1400244D
:101730002A7F2A120062640813230036495522507A
:1017400000000503000000001C22410000004122AF
:101750001C000014083E08140008083E0808000099
:1017600000A0600000080808080800006060000091
:10177000002010080402003E5149453E0000427F0F
:101780004000004261514946002141454B3100185B
:1017900014127F10002745454539003C4A4949301D
:1017A00000017109050300364949493600064949D7
:1017B000291E0000363600000000563600000008E2
:1017C00014224100001414141414000041221408BF
:1017D00000020151090600324959513E007C1211A4
:1017E000127C007F49494936003E41414122007F39
:1017F0004141221C007F49494941007F09090901F3
:10180000003E4149497A007F0808087F0000417F77
:101810004100002040413F01007F08142241007F29
:1018200040404040007F020C027F007F0408107F90
:10183000003E4141413E007F09090906003E4151F9
:10184000215E007F091929460046494949310001B6
:10185000017F0101003F4040403F001F2040201F0A
:10186000003F4038403F00631408146300070870CD
:10187000080700615149454300007F414100005580
:101880002A552A55000041417F000004020102044C
:101890000040404040400000010204000020545439
:1018A0005478007F48444438003844444420003889
:1018B0004444487F00385454541800087E090102FB
:1018C0000018A4A4A47C007F080404780000447DD0
:1018D0004000004080847D00007F1028440000000C
:1018E000417F4000007C04180478007C08040478E0
:1018F00000384444443800FC2424241800182424CC
:1019000018FC007C080404080048545454200004C7
:101910003F444020003C4040207C001C2040201CD4
:10192000003C4030403C004428102844001CA0A04B
:10193000A07C004464544C44141414141414000087
:10194000000000000000000000000000FC0000009B
:10195000000002000000000C020C02000000000069
:10196000000090D0BCD0BC900003000300001824FD
:10197000FE448C000302070201001824D8B04C80FA
:10198000000300010201C038E438E0000102020156
:101990000202080600000000000000000000000035
:1019A00000F80402000000010204000204F8000034
:1019B0000004020100009060F86090000000010047
:1019C00000002020FC20200000000100000000009A
:1019D0000000000008060000000020202020200059
:1019E00000000000000000000000000000020000F5
:1019F00000000080601C0200040300000000F804E6
:101A00000404F8000102020201000008FC000000CA
:101A1000000203020000188444241800030202029A
:101A2000020008042424D80001020202010040B090
:101A300088FC80000000000302003C242424C40031
:101A4000010202020100F824242CC000010202025B
:101A500001000C04E41C0400000003000000D82472
:101A60002424D80001020202010038444444F80052
:101A7000000302020100000010000000000002004C
:101A80000000000020000000000006000000002010
:101A90005088040200000000010290909090900095
:101AA0000000000000000002048850200002010035
:101AB00000001804C4241800000002000000F8040C
:101AC000E494F80001020202020000E09CF08000B1
:101AD00002030000030204FC2424D80002030202D3
:101AE0000100F80404040C0001020202010004FCDD
:101AF0000404F80002030202010004FC24740C0038
:101B000002030202030004FC24740C00020302001E
:101B10000000F0080444CC4000010202010004FC73
:101B20002020FC040203000003020404FC0404005F
:101B3000020203020200000404FC0404060404037D
:101B4000000004FC24D00C0402030200030204FC85
:101B500004000000020302020203FC3CC03CFC0043
:101B600003000300030004FC30C4FC040203020071
:101B70000300F8040404F80001020202010004FC5E
:101B800024241800020302000000F8848404F800F2
:101B900001020207050004FC24649800020302000D
:101BA0000302182424448C000302020201000C04E6
:101BB000FC040C0000020302000004FC0000FC0412
:101BC000000102020100047C80E01C04000003000C
:101BD00000001CE03CE01C00000300030000049C2B
:101BE000609C0400020300030200041CE01C0400CB
:101BF0000002030200000C84641C040002030202C1
:101C000003000000FE020200000007040400000EB2
:101C100030C00000000000010200000202FE0000CF
:101C2000000404070000000402040000000000009B
:101C30000000000000000000080808080808000074
:101C4000020000000000000000000040A0A0C00052
:101C500000010202030204FC2020C0000003020273
:101C6000010000C02020600000010202020000C04C
:101C70002024FC0000010202030200C0A0A0C0005A
:101C80000001020202000020F824240400020302E2
:101C900002000040A0A0602000070A0A0A0404FC19
:101CA0002020C0000203020003020020E400000024
:101CB000000203020000000020E4000008080807FA
:101CC000000004FC80E02020020302000302040460
:101CD000FC000000020203020200E020E020C0003D
:101CE00003000300030020E02020C00002030200E4
:101CF000030200C02020C00000010202010020E019
:101D00002020C000080F0A02010000C02020E000CF
:101D10000001020A0F0820E0402020000203020018
:101D200000000060A0A020000002020203000020CA
:101D3000F820000000000102020020E00020E00086
:101D400000010202030220E0208060200000030165
:101D500000006080E080600000030003000020605D
:101D60008060200002030003020020E02080602049
:101D70000808070100000020A06020000002030204
:101D80000200000020DE0200000000070400000046
:101D900000FF00000000000F00000002DE20000035
:101DA0000004070000000201020404020000000019
:101DB0000000000000000000000000000000000023
:101DC0000000000000F800000000000000333000B8
:101DD000000000100C06100C0600000000000000BF
:101DE000000040C07840C0784000043F04043F0435
:101DF0000400007088FC08300000001820FF211E3D
:101E00000000F008F000E018000000211C031E2173
:101E10001E0000F00888700000001E2123241927EE
:101E2000211010160E00000000000000000000004D
:101E30000000000000E01804020000000007182065
:101E4000400000020418E0000000004020180700D5
:101E50000000404080F0804040000202010F01027B
:101E60000200000000F0000000000101011F01015C
:101E70000100000000000000000080B070000000C1
:101E8000000000000000000000000001010101014D
:101E900001010000000000000000003030000000E0
:101EA00000000000000080601804006018060100B7
:101EB000000000E010080810E000000F10202010C3
:101EC0000F00001010F8000000000020203F20202C
:101ED00000000070080808887000003028242221C3
:101EE0003000003008888848300000182020201179
:101EF0000E000000C02010F8000000070424243F5A
:101F0000240000F808888808080000192120201102
:101F10000E0000E0108888180000000F112020112A
:101F20000E0000380808C83808000000003F000014
:101F300000000070880808887000001C22212122FF
:101F40001C0000E010080810E000000031222211FF
:101F50000F00000000C0C000000000000030300092
:101F60000000000000800000000000008060000011
:101F7000000000008040201008000001020408104A
:101F80002000404040404040400004040404040459
:101F90000400000810204080000000201008040207
:101FA0000100007048080808F00000000030360109
:101FB0000000C030C828E810E000071827242314C8
:101FC0000B000000C038E0000000203C2302022784
:101FD000382008F8888888700000203F20202011D1
:101FE0000E00C0300808080838000718202020100C
:101FF000080008F808080810E000203F2020201002
:102000000F0008F88888E8081000203F20202320CF
:10201000180008F88888E8081000203F2000030016
:102020000000C03008080838000007182020221ED1
:10203000020008F808000008F808203F21010121EB
:102040003F20000808F8080800000020203F20205A
:10205000000000000808F8080800C08080807F00A9
:10206000000008F888C028180800203F2001263802
:10207000200008F8080000000000203F2020202059
:10208000300008F8F800F8F80800203F003F003F53
:10209000200008F830C00008F808203F200007188A
:1020A0003F00E01008080810E0000F10202020106A
:1020B0000F0008F808080808F000203F210101017E
:1020C0000000E01008080810E0000F182424385021
:1020D0004F0008F8888888887000203F2000030C93
:1020E000302000708808080838000038202121229C
:1020F0001C00180808F8080818000000203F2000FD
:10210000000008F808000008F808001F2020202020
:102110001F000878880000C83808000007380E0142
:102120000000F80800F80008F800033C0700073C2E
:102130000300081868808068180820302C03032CDE
:1021400030200838C800C83808000000203F2000B0
:10215000000010080808C838080020382621202070
:102160001800000000FE020202000000007F404054
:102170004000000C30C000000000000000010638E4
:10218000C00000020202FE000000004040407F004C
:102190000000000004020202040000000000000031
:1021A000000000000000000000008080808080802F
:1021B0008080000202040000000000000000000017
:1021C000000000008080808000000019242222226C
:1021D0003F2008F8008080000000003F11202011FF
:1021E0000E000000008080800000000E11202020E2
:1021F0001100000000808088F800000E11202010DF
:102200003F200000808080800000001F22222222C8
:102210001300008080F0888888180020203F20204C
:1022200000000000808080808000006B9494949374
:10223000600008F8008080800000203F210000201E
:102240003F2000809898000000000020203F2020C0
:102250000000000000809898000000C08080807F0F
:10226000000008F8000080808000203F24022D300C
:102270002000000808F8000000000020203F202077
:1022800000008080808080808000203F20003F20F0
:10229000003F8080008080800000203F21000020DF
:1022A0003F200000808080800000001F2020202030
:1022B0001F00808000808000000080FFA12020118E
:1022C0000E000000008080808000000E112020A001
:1022D000FF80808080008080800020203F212000BF
:1022E00001000000808080808000003324242424AA
:1022F0001900008080E0808000000000001F202086
:1023000000008080000000808000001F202020103E
:102310003F20808080000080808000010E30080611
:10232000010080800080008080800F300C030C3022
:102330000F0000808000808080000020312E0E3150
:102340002000808080000080808080818E70180650
:10235000010000808080808080000021302C2221BC
:10236000300000000000807C020200000000003FFE
:10237000404000000000FF00000000000000FF00DF
:1023800000000002027C800000000040403F00008E
:102390000000000601010202040400000000000029
:1023A000000000000000000000000000000000002D
:1023B000000000000000000000000000000000001D
:1023C0000000000000000000000000F0F0F000003D
:1023D00000000000000000017F010000000000007C
:1023E0000000001C1C1C0000000000008060301C6D
:1023F0008C60301C0C000000000000000000000099
:1024000000000000000000000000000000000000CC
:1024100000E00000000000E000000086E69F8686E5
:102420008686E69F860000011F01010101011F0150
:102430000100000080C06020F820E0C00000000023
:1024400003070C18FF70E18100000000070F101057
:102450007F100F0700008060206080000000E020F7
:1024600000000F3020309F70DC371030C0000000BB
:10247000100E03000718101807000000C02020E00D
:10248000C0000000000080E01F38E88703C43C045F
:102490000000070F1810100B070D10100800008027
:1024A0008C4C38000000000000000000000000001C
:1024B000000000000000000000000000000000001C
:1024C000000000000000000080E030080400000070
:1024D000000000FEFF0100000000000000000000FE
:1024E000030F1820400000040830E08000000000C6
:1024F00000000000000001FFFE000000000000409E
:1025000020180F0300000000000000000000000081
:10251000C00000000000004266663C18FF183C66E0
:102520006642000000000000030000000000000000
:1025300000000000800000000000001010101010CB
:10254000FF10101010100000000000000300000039
:10255000000000000000000000000000000000007B
:102560000000000000000000000000808C4C3800DB
:10257000000000000000000000000000000000005B
:1025800000000010101010101010101010000000AB
:10259000000000000000000000000000000000003B
:1025A000000000000000000000000000000000002B
:1025B000000000001C1C1C000000000000000000C7
:1025C000000000000000E0380C00000000008070F7
:1025D0001C03000000000060380E01000000000035
:1025E0000000000080C060202060C080000000FE6D
:1025F000FF010000000001FFFE000001070E18109F
:1026000010180E0701000000808080C0E00000006C
:1026100000000000000000FFFF00000000000000BC
:102620001010101F1F1010100000008040202020EC
:102630002060C080000000030300804020381F0796
:102640000000001C1A1918181818181F0000008024
:10265000C020202060C08000000000030300101094
:10266000182FE780000000070F10101010180F0738
:102670000000000000000000C0E0F000000000C00A
:10268000B088868180FFFF8080000000000000107D
:10269000101F1F1010000000E0606060606060604C
:1026A000000000003F1008080818F0E000000007D4
:1026B0000B101010101C0F030000000080C0402001
:1026C0002020E0C0000000FCFF211008080818F0DE
:1026D000E0000001070C18101010080F03000000A4
:1026E000C0E06060606060E0600000000300000027
:1026F000E0180700000000000000001F1F0000009D
:1027000000000080C0602020202060C08000008782
:10271000EF2C1818303068CF830000070F08101016
:102720001010180F07000000C0C020202020C0801B
:102730000000001F3F604040402010FFFE000000EE
:102740000C1C101010080F03000000000000000017
:1027500000000000000000000000000E0E0E00004F
:10276000000000000000001C1C1C00000000000015
:102770000000000000000000000000000000000C4D
:102780000C000000000000000000005838000000AD
:102790000000000000000000008040201000000049
:1027A000102844820100000000000000000000002A
:1027B00001020408100000000000000000000000FA
:1027C00000000084848484848484848484000000E1
:1027D0000000000000000000000000001020408009
:1027E00000000000000000000000000001824428FA
:1027F000100000001008040201000000000000C0EA
:1028000020201010101030E0C0000003030000F082
:1028100010080C070300000000001C1C1C00000036
:102820000000000000C0406020202040C00000FCEC
:10283000FF01F00E03C1FE03807F0001070E0811A7
:102840001110110904020000000080E0E000000007
:1028500000000000807C4340477FF8800000101893
:102860001F1000000000131F1C1020E0E02020209B
:102870002060C080000000FFFF10101010182FE72C
:102880008000101F1F1010101010180F07000000FC
:1028900080C0402020202060E00000FCFF010000FC
:1028A0000000000001000001070E181010100804BD
:1028B000030020E0E02020202040C080000000FF36
:1028C000FF000000000001FFFE00101F1F1010108D
:1028D00018080E07010020E0E020202020202060C2
:1028E000800000FFFF101010107C00000000101F7F
:1028F0001F10101010101018060020E0E0202020FB
:1029000020206060800000FFFF101010107C00008D
:102910000100101F1F100000000000000000000058
:1029200080C06020202040E0000000FCFF0100008B
:102930004040C0C140400001070E181010100F0F9A
:10294000000020E0E0200000000020E0E02000FF88
:10295000FF101010101010FFFF00101F1F100000BC
:102960000000101F1F100000202020E0E020202089
:1029700000000000000000FFFF0000000000000059
:102980001010101F1F101010000000000000202069
:1029900020E0E020202000000000000000FFFF00F9
:1029A00000000060E0808080C07F3F00000020E0E9
:1029B000E020000020A06020200000FFFF30187CF5
:1029C000E3C000000000101F1F10000001131F1CB7
:1029D000181020E0E020000000000000000000FFD0
:1029E000FF000000000000000000101F1F1010106A
:1029F00010101018060020E0E0E000000000E0E009
:102A0000E02000FF013FFEC0E01E01FFFF00101F9D
:102A10001000031F0300101F1F1020E0E0C0000083
:102A200000000020E02000FF0003071C78E0800089
:102A3000FF00101F100000000000030F1F00000027
:102A400080C060202060C080000000FEFF01000008
:102A5000000000FFFE000001070E181010180C0700
:102A6000010020E0E0202020202060C0800000FF46
:102A7000FF2020202020301F0F00101F1F100000FB
:102A8000000000000000000080C060202060C080C6
:102A9000000000FEFF010000000000FFFE0000013A
:102AA000070E1111133C7C67210020E0E02020205C
:102AB000202060C0800000FFFF101030F0D0080F11
:102AC0000700101F1F10000000030F1C10100080D3
:102AD000C060202020204040E00000070F0C1818A4
:102AE000303060E08100001F0C0810101010180F2B
:102AF00007008060202020E0E0202020608001008E
:102B0000000000FFFF000000000100000000101F97
:102B10001F100000000020E0E02000000000002066
:102B2000E02000FFFF00000000000000FF000007A1
:102B30000F1810101010100807002060E0E02000AF
:102B4000000020E060200000077FF88000807C0308
:102B5000000000000000071F1C070000000020E02C
:102B6000E02000E0E0200020E0200007FFF8E01F68
:102B7000FFFCE01F00000000031F0300011F030013
:102B80000000002060E0A0000020E06020000000C5
:102B900000038F7CF8C6010000000010181E13000F
:102BA00001171F1810002060E0E02000000020E066
:102BB0006020000001073EF8E01807000000000058
:102BC0000010101F1F101000000000806020202047
:102BD00020A0E0E0200000000000C0F03E0F030055
:102BE000000000101C1F1710101010180600000025
:102BF000000000FC0404040404000000000000FFC6
:102C000000000000000000000000007F4040404045
:102C10004000000010E00000000000000000000084
:102C20000000031C608000000000000000000000A5
:102C300000030C70800000000404040404FC000085
:102C4000000000000000000000FF00000000000085
:102C500040404040407F0000000000000010080C91
:102C6000040C08100000000000000000000000003C
:102C70000000000000000000000000000000000054
:102C80000000000000000000000000000000000044
:102C90000000000000008080808080808080808034
:102CA000808000000004040808000000000000000C
:102CB0000000000000000000000000000000000014
:102CC0000000000000000000000000000000000004
:102CD0000000000098D844642424FCF80000000F91
:102CE0001F18101010081F1F10180020E0F000001F
:102CF0000000000000000000FFFF180804040CF8AA
:102D0000F00000001F0F18101010180F0300000033
:102D10000000000000000000000000E0F8180404BB
:102D2000043C3800000000030F0C101010100806BF
:102D300000000000000000000020E0F0000000E0C3
:102D4000F81C04040408FFFF000000030F18101013
:102D500010081F0F08000000000000000000000025
:102D600000000000E0F8484444444C787000000043
:102D7000030F0C181010100804000000000080C0A1
:102D8000602020E0C00000040404FFFF04040404E9
:102D90000000000010101F1F1010100000000000A5
:102DA00000000000000000000000000070F88C042B
:102DB000048CF874040C007076CF8D8D8D89C878E2
:102DC00070000020E0F000000000000000000000A3
:102DD000FFFF08040404FCF8000000101F1F10008F
:102DE00000101F1F100000000000006060000000C5
:102DF00000000000040404FCFC00000000000000CF
:102E00001010101F1F101010000000000000000024
:102E100000606000000000000000040404FCFC00EE
:102E200000000000C0C08080C07F3F000000002084
:102E3000E0F000000000000000000000FFFF80C084
:102E4000F41C0404000000101F1F1100031F1C10BD
:102E500010000000202020E0F00000000000000032
:102E6000000000FFFF000000000000001010101F15
:102E70001F10101000000000000000000000000003
:102E8000000004FCFC0804FCFC0804FCFC00101F0F
:102E90001F10001F1F10001F1F1000000000000067
:102EA0000000000000000004FCFC08080404FCF81A
:102EB000000000101F1F100000101F1F1000000056
:102EC0000000000000000000000000E0F0180C040A
:102ED000040C18F0E00000030F0C101010100C0F81
:102EE00003000000000000000000000000000004DB
:102EF000FCFC080404040CF8F0000080FFFF88903C
:102F000010101C0F03000000000000000000000073
:102F1000000000E0F81C04040408F8FC00000003B2
:102F20000F1810109088FFFF8000000000000000C4
:102F3000000000000000040404FCFC100804040C61
:102F40000C001010101F1F101010000000000000D7
:102F50000000000000000000000000003078CCC439
:102F60008484840C1C0000001E1810101011190F0E
:102F700006000000000000C0000000000000000487
:102F80000404FFFF040404000000000000000F1F01
:102F90001010100C000000000000000000000000F5
:102FA00000000004FCFE00000004FCFE0000000025
:102FB0000F1F181010081F0F08000000000000006D
:102FC00000000000000000040C3CFCC40000C43CF5
:102FD0000C0400000000010F1E0E010000000000A4
:102FE00000000000000000000000043CFCC400E4FD
:102FF0007CFC84807C040000071F070000071F077B
:1030000000000000000000000000000000000004BC
:10301000041C7CE4C0341C0404000010101C1601C5
:10302000131F1C181000000000000000000000002A
:10303000000000040C3CFCC400C43C04040000007C
:10304000C080C1370E010000000000000000000039
:1030500000000000000000001C0404C4F47C1C04F8
:1030600000000000101C1F17111010180E000000A7
:103070000000000000F80C04000000000000001038
:1030800028EF00000000000000000000003F60404A
:103090000000000000000000FF0000000000000031
:1030A00000000000FF000000000000000000000021
:1030B000FF00000000000000040CF8000000000009
:1030C000000000000000EF281000000000000000D9
:1030D00040603F00000000000000001806020204EB
:1030E0000810202030080000000000000000000050
:1030F00000000000000000000000000000000000D0
:1031000000000000000000000000000000000000BF
:1031100000000000000000000000000000000000AF
:10312000000000000000000000000000000000009F
:1036A000000000000000808080808080000000001A
:1036B00000C0E0E0E0E0C0C000000000000000004A
:1036C00000000000000000000000000000000000FA
:1036D00000000000000000000000000000000000EA
:1036E00000000000000000007EFEFEFEFEFEFE0068
:1036F000000080FEFEFEFEFEFEFEFC00000000FC60
:10370000FEFEFEFEFE3E0000000000000000808085
:1037100080808080000000000000000000000000A9
:1037200080F8FEFEFEFEFEFEFEFEF08000000000C1
:103730000000000000000000008080808080800089
:103740000000000000F8F8F8F8F8F8F800000000B1
:10375000000000000000000000000000E0F0F8FCA5
:10376000FCFEFE7E7E3E3E7E7EFEFCFC783000004F
:103770000000F8F8F8F8F8F8F80000000000000081
:103780000000000000000000000000000000000039
:1037900000000000000000000000808080808000A9
:1037A000FFFFFFFFFFFFFF000000030F1F1F1F1F92
:1037B0000F0F00000000000000000080808080806B
:1037C00080800000000000000000000000000000F9
:1037D00000000000000000000000000000000000E9
:1037E0000000003FFFFFFFFFFFFC00C0FFFFFFFFE7
:1037F0007FFFFFFFFFFF8000FEFFFFFFFFFF0F00C7
:103800000000F0F8FEFEFFFF7F1F0F0F1FFFFFFFFE
:10381000FEFCF8C000000000C0FCFFFFFFFF7F07B8
:103820001FFFFFFFFFFFF88000000000C0F0FCFE5C
:10383000FFFFFF7F1F1F1F1F3F3F3F0E041F1FFF84
:10384000FFFFFFFFFFFF1F1F1F1F00000000000002
:103850000000000000001F7FFFFFFFFFFFFCF8F8E3
:10386000F0F0E0E0C1C08000001F1F1FFFFFFFFF5E
:10387000FFFFFF1F1F1F0F000000FFFFFFFFFFFFE5
:1038800000000000FFFFFFFFFFFFFF000000C0F887
:10389000FCFEFFFFFF7F1F1F1F3FFFFFFFFFFFFF1C
:1038A000FF00000000FFFFFFFFFFFFFF000000C060
:1038B000F8FCFEFFFFFF3F1F1F1F3FFFFFFFFEFC47
:1038C000F8E0000000000000000000000000000020
:1038D00000000000000000000000000000000FFFDA
:1038E000FFFFFFFFFCFFFFFFFF1F0001FFFFFFFFC8
:1038F000FFFEFFFFFFFFFF070000001EFFFFFFFFAF
:10390000FFFFDF1F1F1F1F1F1F9F9F1F1F1F000085
:10391000E0FEFFFFFFFFFFFFFCFCFCFDFFFFFFFFE2
:10392000FFFFFCC00000FFFFFFFFFFFFFF80000064
:10393000000000800000000000FFFFFFFFFFFFFF0E
:103940000000000000000000000000000000000077
:1039500080C0C0800101030303070FFFFFFFFFFFCB
:10396000FFFF70000000FFFFFFFFFFFFFF000000F0
:1039700000000000FFFFFFFFFFFF00000080FFFFCF
:10398000FFFFFFFFFF000000FFFFFFFFFFFFFF80C3
:1039900000000000FFFFFFFFFFFFFF00000000FF2F
:1039A000FFFFFFFFFFFF000000FFFFFFFFFFFFFF24
:1039B0008000000000FFFFFFFFFFFFFF000000008E
:1039C00000000000000000000000000000000000F7
:1039D000000000000000000000073F3F3F3F3F3F66
:1039E0003F3F0F000000003F3F3F3F3F3F3F3F3F13
:1039F00001000000000001070F1F1F3F3F3F3E3E38
:103A00003E3E3F3F1F1F0E00303E3F3F3F3F3F1FA8
:103A100001000000000000033F3F3F3F3F3F3C00EC
:103A20000003070F1F3F3F3F3F3E3E3F3F3F1F1EEC
:103A3000080000030F1F3F3F3F3F3F3E3F3F1C1822
:103A4000000000000000000000070F1F1F3F3F3F65
:103A50003F3E3E3F3F3F3F1F1F0F07030000000058
:103A6000070F1F3F3F3F3F3E3F3F3F1C00000F1FE0
:103A70003F3F3F3F3F3E3F1F1F3F3F3F3F3F3F00D6
:103A8000000000070F1F3F3F3F3F3F3E3F1F1F3FCC
:103A90003F3F3F3F3F000000003F3F3F3F3F3F3F32
:103AA0000000000003070F1F3F3F3F3F3E3E3F3FE8
:103AB0003F1F1F0F03000000000000000000000077
:103AC00000000000000000000000000000000000F6
:103AD00000000000000000000000000000000000E6
:103AE00000000000000000000000000000000000D6
:103AF00000000000000000000000000000000000C6
:1041C0000000000000000000000000000000C0C06F
:1041D000C0C0C0000080C0C0C0C08000000000009F
:1041E00000000000000000000000000000000000CF
:1041F00000000000000000000000000000000000BF
:1042000000000000000000000000000000000000AE
:10421000000000000000000000000000000000009E
:10422000000000000000000000000000000000008E
:10423000000000000000000000000000000000007E
:10424000000000000000000000000000000000006E
:10425000000000000000000000000000000000005E
:1042600000C0C0C0C0C0C0000000000000000000CE
:1042700000000000000000C0C0C0C0C0000000007E
:10428000000000000000000000000000000000002E
:1042900000000000000000000000000C1E1F1F0FA7
:1042A0000F9FFFFFFEFEF8000000000000003878BE
:1042B0007C7E3EFFFFFFFFFF00040E1E1F8F8F8FCF
:1042C000FFFFFFFEFC000000737F3F1F0F00003167
:1042D0007B7F3F1F070000000000000000FFFFFF82
:1042E000FFFF8787878787070000F0F0F0F0F0F086
:1042F00070F8F8F0F0E0800030F0F0F07878F8F046
:10430000F0F0E0800000F0F0F0F0F0F070F8F8F07D
:10431000F0E0800080E0F0F0F0F878F0F0F0E0C03D
:104320000000F0F0F0F0F0F0F0F0F010000000000D
:10433000000000FFFFFFFFFFFFFEC0E0FFFFFFFFE9
:10434000FFFFFF000080C0E0F0F0F078F8F0F0F040
:10435000E0C00000C0E0F0F0F8F870FFFFFFFFFFE2
:10436000FF0000F0F0F0F0F000F0F0F0F0F0F000FE
:1043700000FFFFFFFFFF000080C0E0F0F0F878F8DA
:10438000F0F0F0E0800000000000000000000000FD
:10439000000000000080C0F0F8FCFEFFBF9F878394
:1043A0008000C0C0C0C0C0800000000000FFFFFF50
:1043B000FFFF0080C0C0C0C78787CFFFFFFFFEF8A8
:1043C00000000000000000000000000000000000ED
:1043D00000000000000000FFFFFFFFFF87878787C6
:1043E00087800000FFFFFFFFFF8080E1FFFFFFFFEE
:1043F0007F40F8FCFCFEFE9ECFFFFFFFFFFF0000AA
:10440000FFFFFFFFFF8080E1FFFFFFFF7F00FFFF57
:10441000FFFFFFDC9C9D9FDFDF9F1F00FFFFFFFF73
:10442000FF0301000000000000000000FFFFFFFF8D
:10443000FF0FFFFFFFFFFFFF0FFFFFFFFFFC007FEE
:10444000FFFFFFFFE18080FFFFFFFFFF1C08FFFF72
:10445000FFFFFF8080FFFFFFFFFFFF0000FFFFFF68
:10446000FFFF80FFFFFFFFFFFF0000FFFFFFFFFFD9
:1044700080007FFFFFFFFFDC9C9C9FDFDF9F1F0012
:104480000000000000000000000000000000000725
:1044900007070707070707070707070003070707B7
:1044A00007030000000000070707070700010303D8
:1044B00007070707070707030100000000000000C7
:1044C00000000000000000000000000000000000EC
:1044D0000007070707070707070707070000FFFF91
:1044E000FFFFFF0707070707030100000307070790
:1044F00007070703070707070000FFFFFFFFFF0786
:104500000707070703010000000103070707070764
:104510000707030300000707070707000000000064
:104520000000000000000707070707000101010164
:104530000100000707070707000001030707070737
:104540000707070303000000010307070707070722
:1045500007070707070000030707070707070707FD
:1045600007070700000307070707070700010307FE
:10457000070707070707030300000000000000000B
:10458000000000000000000000000000000000002B
:10459000000000000000000000000000000000001B
:1045A000000000000000000000000000000000000B
:1045B00000000000000000000000000000000000FB
:104B9000000070F0F8FC7CFEFEFEFEFE00183C3CBF
:104BA0003E3E1E1EFEFEFEFCF800183C3E3E1E1E53
:104BB0003EFEFEFCFCF000000000000000E0E0E033
:104BC000E0E0C080E0E0E0E0E0000000000000186D
:104BD0003C3C3E3E1E1EFEFEFEFCF80000FEFEFEBD
:104BE000FEFE9E9E9E9E1E1E0000E0F8FCFEFE7EC7
:104BF0001E3EFEFEFCF8E00000000000000000FE8B
:104C0000FEFEFEFEFE0E0E0E0E0E0E00000000005A
:104C100000000000000000FEFEFEFEFE000000009E
:104C2000000000FEFEFEFEFE000000FEFEFEFEFE98
:104C3000FEFCE000FEFEFEFEFE0000FEFEFEFEFEAE
:104C4000C0E0F8FCFEFE3E1E060000000000000072
:104C50000000000000000000000000000000000054
:104C60000000000000000000000000000000000044
:104C70000000000000000000000000000000000034
:104C80000000000000000000000000000000000024
:104C900000FFFFFFFFFF000080C0E0F0FCFE7F3F51
:104CA0001F0F03000080E0F0F8FCFF7F3F0F0701BB
:104CB0000000000000000000C1E7FFFFFFFFFFFF52
:104CC000F7C1000000000000000080C0E0F0FCFE22
:104CD0007F3F1F0F0300008787878707078FFFFF2E
:104CE000FFFFFC007FFFFFFFFFC00080FFFFFFFF13
:104CF000FF0000000000000000FFFFFFFFFFFF0FAC
:104D00000F0F0F0F00001E1E1E1E1E1E1E1E1E0059
:104D100000FFFFFFFFFF00000000000000FFFFFF9B
:104D2000FFFF000000FFFFFFFFFF3FFFFFFFFFFF50
:104D3000FFFFFF0000FFFFFFFFFF1F7FFFFFFFF8E8
:104D4000E0C00000000000000000000000000000C3
:104D50000000000000000000000000000000000053
:104D60000000000000000000000000000000000043
:104D70000000000000000000000000000000000033
:104D800000000000000000000000000F0F0F0F0FD8
:104D900000000F0F0F0F0F0F0F0F0F0F0F070F0F49
:104DA0000F0F0F0F0F0F0F0F0F0F0000000000006D
:104DB0000C0F0F0F0F0F0101070F0F0F0F0C00004B
:104DC000000000000F0F0F0F0F0F0F0F0F0F0F0737
:104DD0000307070F0F0F0F0F0F0F0703010000034B
:104DE000070F0F0F0F0F0F0F070300000000000049
:104DF0000000000F0F0F0F0F0F0F0F0F0F0F0F00FF
:104E000000000000000000000000000F0F0F0F0F57
:104E10000F0F0F0F0F0F000F0F0F0F0F0000000FDE
:104E20000F0F0F0F00010F0F0F0F0F0F0F00000FCD
:104E30000F0F0F0F000001030F0F0F0F0F0C0000DB
:104E40000000000000000000000000000000000062
:104E50000000000000000000000000000000000052
:104E60000000000000000000000000000000000042
:104E70000000000000000000000000000000000032
:104E80000000000000000000000000000000000022
:104E90000000000000000000000000000000000012
:104EA0000000000000000000000000000000000002
:104EB00000000000000000000000000000000000F2
:104EC00000000000000000000000000000000000E2
:104ED00000000000000000000000000000000000D2
:104EE00000000000000000000000000000000000C2
:104EF00000000000000000000000000000000000B2
:104F000000000000000000000000000000000000A1
:104F10000000000000000000000000000000000091
:104F20000000000000000000000000000000000081
:104F30000000000000000000000000000000000071
:104F40000000000000000000000000000000000061
:104F50000000000000000000000000000000000051
:104F60000000000000000000000000000000000041
:104F70000000000000000000000000000000000031
:104F80000000000000000000000000000000000021
:104F90000000000000000000000000000000000011
:104FA0000000000000000000000000000000000001
:104FB00000000000000000000000000000000000F1
:104FC00000000000000000000000000000000000E1
:104FD00000000000000000000000000000000000D1
:104FE00000000000000000000000000000000000C1
:104FF00000000000000000000000000000000000B1
:1050000000000000000000000000000000000000A0
:105010000000000000000000000000000000000090
:105020000000000000000000000000000000000080
:105030000000000000000000000000000000000070
:10504000605000080000002008000000C0010008B7
:105050006850000808000020C0250000DC0100089E
:085060000100000000127A00BB
:040000050800018569
:00000001FF
